BL51 BANKED LINKER/LOCATER V6.22                                                        08/01/2023  15:41:50  PAGE 1


BL51 BANKED LINKER/LOCATER V6.22, INVOKED BY:
D:\KEIL\C51\BIN\BL51.EXE .\Objects\STARTUP.obj, .\Objects\GPIO.obj, .\Objects\Initial.obj, .\Objects\main.obj, .\Objects
>> \TouchKeyScan.obj, .\User\C\XC8FT8463_Touch_V1.1.LIB TO .\Objects\XC8FT8463 PRINT (.\Listings\XC8FT8463.m51) RAMSIZE 
>> (256)


MEMORY MODEL: SMALL


INPUT MODULES INCLUDED:
  .\Objects\STARTUP.obj (?C_STARTUP)
  .\Objects\GPIO.obj (GPIO)
  .\Objects\Initial.obj (INITIAL)
  .\Objects\main.obj (MAIN)
  .\Objects\TouchKeyScan.obj (TOUCHKEYSCAN)
  .\User\C\XC8FT8463_Touch_V1.1.LIB (TOUCH_LIB)
  D:\KEIL\C51\LIB\C51S.LIB (?C_INIT)
  D:\KEIL\C51\LIB\C51S.LIB (?C?CLDPTR)
  D:\KEIL\C51\LIB\C51S.LIB (?C?CLDOPTR)
  D:\KEIL\C51\LIB\C51S.LIB (?C?CILDOPTR)
  D:\KEIL\C51\LIB\C51S.LIB (?C?CSTPTR)
  D:\KEIL\C51\LIB\C51S.LIB (?C?CSTOPTR)
  D:\KEIL\C51\LIB\C51S.LIB (?C?SIDIV)
  D:\KEIL\C51\LIB\C51S.LIB (?C?ILDOPTR)
  D:\KEIL\C51\LIB\C51S.LIB (?C?IILDOPTR)
  D:\KEIL\C51\LIB\C51S.LIB (?C?ISTPTR)
  D:\KEIL\C51\LIB\C51S.LIB (?C?ISTOPTR)
  D:\KEIL\C51\LIB\C51S.LIB (?C?LMUL)
  D:\KEIL\C51\LIB\C51S.LIB (?C?ULDIV)
  D:\KEIL\C51\LIB\C51S.LIB (?C?ULCMP)
  D:\KEIL\C51\LIB\C51S.LIB (?C?ULSHR)
  D:\KEIL\C51\LIB\C51S.LIB (?C?LSHL)
  D:\KEIL\C51\LIB\C51S.LIB (?C?LLDPTR)
  D:\KEIL\C51\LIB\C51S.LIB (?C?LLDOPTR)
  D:\KEIL\C51\LIB\C51S.LIB (?C?LSTPTR)
  D:\KEIL\C51\LIB\C51S.LIB (?C?LSTOPTR)
  D:\KEIL\C51\LIB\C51S.LIB (?C?LLDPTR0)
  D:\KEIL\C51\LIB\C51S.LIB (?C?LLDOPTR0)
  D:\KEIL\C51\LIB\C51S.LIB (?C?LSTKOPTR)
  D:\KEIL\C51\LIB\C51S.LIB (?C?OFFXADD)
  D:\KEIL\C51\LIB\C51S.LIB (?C?LIMUL)
  D:\KEIL\C51\LIB\C51S.LIB (?C?UIDIV)
  D:\KEIL\C51\LIB\C51S.LIB (?C?IILDX)
  D:\KEIL\C51\LIB\C51S.LIB (?C?LLDIDATA)
  D:\KEIL\C51\LIB\C51S.LIB (?C?LLDXDATA)
  D:\KEIL\C51\LIB\C51S.LIB (?C?LLDPDATA)
  D:\KEIL\C51\LIB\C51S.LIB (?C?LLDCODE)
  D:\KEIL\C51\LIB\C51S.LIB (?C?LLDIDATA0)
  D:\KEIL\C51\LIB\C51S.LIB (?C?LLDXDATA0)
  D:\KEIL\C51\LIB\C51S.LIB (?C?LLDPDATA0)
  D:\KEIL\C51\LIB\C51S.LIB (?C?LLDCODE0)
  D:\KEIL\C51\LIB\C51S.LIB (?C?LSTIDATA)
  D:\KEIL\C51\LIB\C51S.LIB (?C?LSTXDATA)
  D:\KEIL\C51\LIB\C51S.LIB (?C?LSTPDATA)
  D:\KEIL\C51\LIB\C51S.LIB (?C?LSTKIDATA)
  D:\KEIL\C51\LIB\C51S.LIB (?C?LSTKXDATA)
  D:\KEIL\C51\LIB\C51S.LIB (?C?LSTKPDATA)

BL51 BANKED LINKER/LOCATER V6.22                                                      08/01/2023  15:41:50  PAGE 2



LINK MAP OF MODULE:  .\Objects\XC8FT8463 (?C_STARTUP)


            TYPE    BASE      LENGTH    RELOCATION   SEGMENT NAME
            -----------------------------------------------------

            * * * * * * *   D A T A   M E M O R Y   * * * * * * *
            REG     0000H     0008H     ABSOLUTE     "REG BANK 0"
            DATA    0008H     0021H     UNIT         _DATA_GROUP_
            DATA    0029H     0020H     UNIT         ?DT?TOUCH_LIB
            IDATA   0049H     0001H     UNIT         ?STACK

            * * * * * * *  X D A T A   M E M O R Y  * * * * * * *
            XDATA   0000H     0218H     UNIT         ?XD?TOUCHKEYSCAN

            * * * * * * *   C O D E   M E M O R Y   * * * * * * *
            CODE    0000H     0003H     ABSOLUTE     
            CODE    0003H     002FH     UNIT         ?PR?_TKL_KEY_CHECKERROR?TOUCH_LIB
                    0032H     0001H                  *** GAP ***
            CODE    0033H     0003H     ABSOLUTE     
            CODE    0036H     0026H     UNIT         ?PR?TKL_CSDINIT?TOUCH_LIB
            CODE    005CH     0007H     UNIT         ?PR?WDT_IRQ?TOUCHKEYSCAN
            CODE    0063H     0003H     ABSOLUTE     
            CODE    0066H     001CH     UNIT         ?PR?SYSTEM_INIT?INITIAL
                    0082H     0009H                  *** GAP ***
            CODE    008BH     0003H     ABSOLUTE     
            CODE    008EH     059FH     UNIT         ?C?LIB_CODE
            CODE    062DH     0275H     UNIT         ?PR?_THRESHOLDINIT?TOUCH_LIB
            CODE    08A2H     025CH     UNIT         ?PR?_TKL_KEY_FINDICOMTREATMENT?TOUCH_LIB
            CODE    0AFEH     0240H     UNIT         ?C_INITSEG
            CODE    0D3EH     023BH     UNIT         ?PR?TKL_ECS?TOUCH_LIB
            CODE    0F79H     0210H     UNIT         ?PR?_GPIO_SET_MODE?TOUCH_LIB
            CODE    1189H     01D3H     UNIT         ?PR?_TKL_INIT?TOUCH_LIB
            CODE    135CH     0185H     UNIT         ?PR?_TKL_ACQUISITION?TOUCH_LIB
            CODE    14E1H     0173H     UNIT         ?PR?TKL_WATERPROOF?TOUCH_LIB
            CODE    1654H     013CH     UNIT         ?PR?_TKL_KEY_PREDETECTEDTREATMENT?TOUCH_LIB
            CODE    1790H     0135H     UNIT         ?PR?_TKL_KEY_POSTDETECTEDTREATMENT?TOUCH_LIB
            CODE    18C5H     0113H     UNIT         ?PR?_TKL_ADDDATATOBUF?TOUCH_LIB
            CODE    19D8H     00CAH     UNIT         ?PR?TKL_GETKEYVALUE?TOUCH_LIB
            CODE    1AA2H     00B8H     UNIT         ?PR?TKL_PROCESSALL?TOUCH_LIB
            CODE    1B5AH     00ABH     UNIT         ?PR?_TKL_KEY_SETIDLESTATE?TOUCH_LIB
            CODE    1C05H     00A7H     UNIT         ?PR?_TKL_SCAN?TOUCH_LIB
            CODE    1CACH     00A6H     UNIT         ?PR?_TKL_KEY_CALIBRATIONTREATMENT?TOUCH_LIB
            CODE    1D52H     00A2H     UNIT         ?PR?_TKL_KEY_DETECTEDTREATMENT?TOUCH_LIB
            CODE    1DF4H     009AH     UNIT         ?PR?_TKL_KEY_SETFINDICOMSTATE?TOUCH_LIB
            CODE    1E8EH     0099H     UNIT         ?PR?_TKL_KEY_IDLETREATMENT?TOUCH_LIB
            CODE    1F27H     0091H     UNIT         ?PR?TKL_SCANSTARTLOOP?TOUCH_LIB
            CODE    1FB8H     0090H     UNIT         ?PR?_TKL_KEY_SETDETECTSTATE?TOUCH_LIB
            CODE    2048H     008FH     UNIT         ?PR?TKL_IRQCALLBACK?TOUCH_LIB
            CODE    20D7H     008CH     UNIT         ?C_C51STARTUP
            CODE    2163H     007CH     UNIT         ?PR?KEYPROCESS?MAIN
            CODE    21DFH     0073H     UNIT         ?PR?_TKL_KEY_SETCALIBRATIONSTATE?TOUCH_LIB
            CODE    2252H     0070H     UNIT         ?PR?_TKL_KEY_SETPRECALIBRATIONSTATE?TOUCH_LIB
            CODE    22C2H     006DH     UNIT         ?PR?_TKL_KEY_PRECALIBRATIONTREATMENT?TOUCH_LIB
            CODE    232FH     006AH     UNIT         ?PR?MAIN?MAIN
            CODE    2399H     0068H     UNIT         ?CO?TOUCHKEYSCAN
BL51 BANKED LINKER/LOCATER V6.22                                                      08/01/2023  15:41:50  PAGE 3


            CODE    2401H     005FH     UNIT         ?PR?_TKL_KEY_SETERRORSTATE?TOUCH_LIB
            CODE    2460H     0058H     UNIT         ?PR?INITIAL_TRIM?INITIAL
            CODE    24B8H     0053H     UNIT         ?PR?_TKL_KEY_DELTACACULATION?TOUCH_LIB
            CODE    250BH     0052H     UNIT         ?PR?GPIO_INIT?GPIO
            CODE    255DH     0044H     UNIT         ?PR?TIMER0_IRQHANDLER?TOUCHKEYSCAN
            CODE    25A1H     003BH     UNIT         ?PR?CSD_IRQHANDLER?TOUCHKEYSCAN
            CODE    25DCH     0035H     UNIT         ?PR?_TKL_KEY_SETPREDETECTSTATE?TOUCH_LIB
            CODE    2611H     0032H     UNIT         ?PR?_DELAY?TOUCH_LIB
            CODE    2643H     0032H     UNIT         ?PR?TKL_ACQUISITIONALL?TOUCH_LIB
            CODE    2675H     0031H     UNIT         ?PR?_TKL_KEY_SETPOSTDETECTSTATE?TOUCH_LIB
            CODE    26A6H     001AH     UNIT         ?PR?_DELAYMS?INITIAL
            CODE    26C0H     0018H     UNIT         ?PR?TKL_ACTION?TOUCH_LIB
            CODE    26D8H     0017H     UNIT         ?PR?_TKL_KEY_BACKIDLESTATE?TOUCH_LIB
            CODE    26EFH     0017H     UNIT         ?PR?_TKL_KEY_BACKTODETECTSTATE?TOUCH_LIB
            CODE    2706H     0010H     UNIT         ?PR?TIMER0_INIT?TOUCHKEYSCAN
            CODE    2716H     0010H     UNIT         ?PR?WDT_INIT?TOUCH_LIB



OVERLAY MAP OF MODULE:   .\Objects\XC8FT8463 (?C_STARTUP)


SEGMENT                                            DATA_GROUP 
  +--> CALLED SEGMENT                            START    LENGTH
----------------------------------------------------------------
?C_C51STARTUP                                    -----    -----
  +--> ?PR?MAIN?MAIN
  +--> ?C_INITSEG

?PR?MAIN?MAIN                                    0008H    0001H
  +--> ?PR?SYSTEM_INIT?INITIAL
  +--> ?PR?GPIO_INIT?GPIO
  +--> ?PR?TIMER0_INIT?TOUCHKEYSCAN
  +--> ?CO?TOUCHKEYSCAN
  +--> ?PR?_TKL_INIT?TOUCH_LIB
  +--> ?PR?_DELAYMS?INITIAL
  +--> ?PR?TKL_ACTION?TOUCH_LIB
  +--> ?PR?KEYPROCESS?MAIN

?PR?SYSTEM_INIT?INITIAL                          -----    -----
  +--> ?PR?_DELAYMS?INITIAL
  +--> ?PR?INITIAL_TRIM?INITIAL

?PR?_TKL_INIT?TOUCH_LIB                          0009H    0014H
  +--> ?PR?_THRESHOLDINIT?TOUCH_LIB
  +--> ?PR?WDT_INIT?TOUCH_LIB
  +--> ?PR?TKL_CSDINIT?TOUCH_LIB
  +--> ?PR?_TKL_KEY_SETFINDICOMSTATE?TOUCH_LIB
  +--> ?PR?_TKL_KEY_FINDICOMTREATMENT?TOUCH_LIB

?PR?_THRESHOLDINIT?TOUCH_LIB                     001DH    0004H

?PR?_TKL_KEY_SETFINDICOMSTATE?TOUCH_LIB          001DH    0001H

?PR?_TKL_KEY_FINDICOMTREATMENT?TOUCH_LIB         001DH    0007H
  +--> ?PR?_TKL_SCAN?TOUCH_LIB
  +--> ?PR?_TKL_KEY_SETCALIBRATIONSTATE?TOUC...
BL51 BANKED LINKER/LOCATER V6.22                                                      08/01/2023  15:41:50  PAGE 4


  +--> ?PR?_TKL_KEY_SETERRORSTATE?TOUCH_LIB

?PR?_TKL_SCAN?TOUCH_LIB                          0024H    0003H
  +--> ?PR?_GPIO_SET_MODE?TOUCH_LIB

?PR?_TKL_KEY_SETCALIBRATIONSTATE?TOUC...         0024H    0001H

?PR?_TKL_KEY_SETERRORSTATE?TOUCH_LIB             0024H    0001H

?PR?TKL_ACTION?TOUCH_LIB                         -----    -----
  +--> ?PR?TKL_ACQUISITIONALL?TOUCH_LIB
  +--> ?PR?TKL_PROCESSALL?TOUCH_LIB
  +--> ?PR?TKL_WATERPROOF?TOUCH_LIB
  +--> ?PR?TKL_ECS?TOUCH_LIB

?PR?TKL_ACQUISITIONALL?TOUCH_LIB                 0009H    0001H
  +--> ?PR?_TKL_ACQUISITION?TOUCH_LIB

?PR?_TKL_ACQUISITION?TOUCH_LIB                   000AH    0013H

?PR?TKL_PROCESSALL?TOUCH_LIB                     0009H    0001H
  +--> ?PR?_TKL_KEY_DELTACACULATION?TOUCH_LIB
  +--> ?PR?_TKL_KEY_CHECKERROR?TOUCH_LIB
  +--> ?PR?_TKL_KEY_IDLETREATMENT?TOUCH_LIB
  +--> ?PR?_TKL_KEY_PREDETECTEDTREATMENT?TOU...
  +--> ?PR?_TKL_KEY_DETECTEDTREATMENT?TOUCH_LIB
  +--> ?PR?_TKL_KEY_POSTDETECTEDTREATMENT?TO...
  +--> ?PR?_TKL_KEY_PRECALIBRATIONTREATMENT?...
  +--> ?PR?_TKL_KEY_SETERRORSTATE?TOUCH_LIB
  +--> ?PR?_TKL_KEY_CALIBRATIONTREATMENT?TOU...
  +--> ?PR?_TKL_KEY_SETIDLESTATE?TOUCH_LIB

?PR?_TKL_KEY_DELTACACULATION?TOUCH_LIB           000AH    0001H

?PR?_TKL_KEY_IDLETREATMENT?TOUCH_LIB             000AH    0001H
  +--> ?PR?_TKL_KEY_SETPRECALIBRATIONSTATE?T...
  +--> ?PR?_TKL_KEY_SETPREDETECTSTATE?TOUCH_LIB

?PR?_TKL_KEY_SETPRECALIBRATIONSTATE?T...         000BH    0001H

?PR?_TKL_KEY_SETPREDETECTSTATE?TOUCH_LIB         000BH    0001H

?PR?_TKL_KEY_PREDETECTEDTREATMENT?TOU...         000AH    0005H
  +--> ?PR?_TKL_KEY_SETDETECTSTATE?TOUCH_LIB
  +--> ?PR?_TKL_KEY_BACKIDLESTATE?TOUCH_LIB
  +--> ?PR?_TKL_KEY_SETIDLESTATE?TOUCH_LIB

?PR?_TKL_KEY_SETDETECTSTATE?TOUCH_LIB            000FH    0001H

?PR?_TKL_KEY_SETIDLESTATE?TOUCH_LIB              000FH    0001H

?PR?_TKL_KEY_DETECTEDTREATMENT?TOUCH_LIB         000AH    0001H
  +--> ?PR?_TKL_KEY_SETPOSTDETECTSTATE?TOUCH...
  +--> ?PR?_TKL_KEY_SETCALIBRATIONSTATE?TOUC...

?PR?_TKL_KEY_SETPOSTDETECTSTATE?TOUCH...         000BH    0001H

BL51 BANKED LINKER/LOCATER V6.22                                                      08/01/2023  15:41:50  PAGE 5


?PR?_TKL_KEY_POSTDETECTEDTREATMENT?TO...         000AH    0005H
  +--> ?PR?_TKL_KEY_BACKTODETECTSTATE?TOUCH_LIB
  +--> ?PR?_TKL_KEY_SETIDLESTATE?TOUCH_LIB

?PR?_TKL_KEY_PRECALIBRATIONTREATMENT?...         000AH    0001H
  +--> ?PR?_TKL_KEY_SETCALIBRATIONSTATE?TOUC...
  +--> ?PR?_TKL_KEY_BACKIDLESTATE?TOUCH_LIB

?PR?_TKL_KEY_CALIBRATIONTREATMENT?TOU...         000AH    0001H
  +--> ?PR?_TKL_KEY_SETIDLESTATE?TOUCH_LIB

?PR?TKL_WATERPROOF?TOUCH_LIB                     0009H    0008H

?PR?TKL_ECS?TOUCH_LIB                            0009H    0007H

?PR?KEYPROCESS?MAIN                              0009H    0004H
  +--> ?PR?TKL_GETKEYVALUE?TOUCH_LIB

?PR?TKL_GETKEYVALUE?TOUCH_LIB                    -----    -----
  +--> ?PR?_DELAY?TOUCH_LIB

*** NEW ROOT ***************************************************

?PR?TIMER0_IRQHANDLER?TOUCHKEYSCAN               -----    -----
  +--> ?PR?TKL_SCANSTARTLOOP?TOUCH_LIB

*** NEW ROOT ***************************************************

?PR?CSD_IRQHANDLER?TOUCHKEYSCAN                  -----    -----
  +--> ?PR?TKL_IRQCALLBACK?TOUCH_LIB

?PR?TKL_IRQCALLBACK?TOUCH_LIB                    -----    -----
  +--> ?PR?_GPIO_SET_MODE?TOUCH_LIB
  +--> ?PR?_TKL_ADDDATATOBUF?TOUCH_LIB

?PR?_TKL_ADDDATATOBUF?TOUCH_LIB                  0027H    0002H



SYMBOL TABLE OF MODULE:  .\Objects\XC8FT8463 (?C_STARTUP)

  VALUE           TYPE          NAME
  ----------------------------------

  -------         MODULE        ?C_STARTUP
  C:20D7H         SEGMENT       ?C_C51STARTUP
  I:0049H         SEGMENT       ?STACK
  C:0000H         PUBLIC        ?C_STARTUP
  D:00E0H         SYMBOL        ACC
  D:00F0H         SYMBOL        B
  D:0083H         SYMBOL        DPH
  D:0082H         SYMBOL        DPL
  N:0000H         SYMBOL        IBPSTACK
  N:0100H         SYMBOL        IBPSTACKTOP
  N:0080H         SYMBOL        IDATALEN
  C:20DAH         SYMBOL        IDATALOOP
  N:0000H         SYMBOL        PBPSTACK
BL51 BANKED LINKER/LOCATER V6.22                                                      08/01/2023  15:41:50  PAGE 6


  N:0100H         SYMBOL        PBPSTACKTOP
  N:0000H         SYMBOL        PDATALEN
  N:0000H         SYMBOL        PDATASTART
  N:0000H         SYMBOL        PPAGE
  N:0000H         SYMBOL        PPAGEENABLE
  D:00A0H         SYMBOL        PPAGE_SFR
  D:0081H         SYMBOL        SP
  C:20D7H         SYMBOL        STARTUP1
  N:0000H         SYMBOL        XBPSTACK
  N:0000H         SYMBOL        XBPSTACKTOP
  N:0000H         SYMBOL        XDATALEN
  N:0000H         SYMBOL        XDATASTART
  C:0000H         LINE#         126
  C:20D7H         LINE#         133
  C:20D9H         LINE#         134
  C:20DAH         LINE#         135
  C:20DBH         LINE#         136
  C:20DDH         LINE#         185
  C:20E0H         LINE#         196
  -------         ENDMOD        ?C_STARTUP

  -------         MODULE        GPIO
  C:0000H         SYMBOL        _ICE_DUMMY_
  D:00A8H         PUBLIC        IE
  C:250BH         PUBLIC        GPIO_Init
  D:00E0H         PUBLIC        ACC
  D:00F8H         PUBLIC        SLPTIM_CR
  D:0080H         PUBLIC        P0_DR
  D:0090H         PUBLIC        P1_DR
  D:00A0H         PUBLIC        P2_DR
  D:00B0H         PUBLIC        P3_DR
  D:00D0H         PUBLIC        PSW
  -------         PROC          GPIO_INIT
  C:250BH         LINE#         11
  C:250BH         LINE#         12
  C:250BH         LINE#         20
  C:2510H         LINE#         21
  C:2516H         LINE#         22
  C:2519H         LINE#         23
  C:251BH         LINE#         24
  C:251DH         LINE#         25
  C:2521H         LINE#         27
  C:2525H         LINE#         28
  C:252BH         LINE#         29
  C:252EH         LINE#         30
  C:2530H         LINE#         31
  C:2532H         LINE#         32
  C:2536H         LINE#         34
  C:253AH         LINE#         35
  C:2540H         LINE#         36
  C:2543H         LINE#         37
  C:2545H         LINE#         38
  C:2547H         LINE#         39
  C:254BH         LINE#         41
  C:2551H         LINE#         42
  C:2554H         LINE#         43
  C:2556H         LINE#         44
BL51 BANKED LINKER/LOCATER V6.22                                                      08/01/2023  15:41:50  PAGE 7


  C:2558H         LINE#         45
  C:255CH         LINE#         46
  -------         ENDPROC       GPIO_INIT
  -------         ENDMOD        GPIO

  -------         MODULE        INITIAL
  C:0000H         SYMBOL        _ICE_DUMMY_
  C:0066H         PUBLIC        System_Init
  D:00A8H         PUBLIC        IE
  D:0095H         PUBLIC        PCLK_CR
  C:26A6H         PUBLIC        _DelayMs
  D:00E0H         PUBLIC        ACC
  D:0094H         PUBLIC        CLK_CR
  D:00F8H         PUBLIC        SLPTIM_CR
  C:2460H         PUBLIC        Initial_trim
  D:0080H         PUBLIC        P0_DR
  D:0090H         PUBLIC        P1_DR
  D:00A0H         PUBLIC        P2_DR
  D:00B0H         PUBLIC        P3_DR
  D:00D0H         PUBLIC        PSW
  -------         PROC          _DELAYMS
  D:0006H         SYMBOL        ms
  -------         DO            
  D:0004H         SYMBOL        a
  -------         ENDDO         
  C:26A6H         LINE#         9
  C:26A6H         LINE#         10
  C:26A6H         LINE#         12
  C:26AAH         LINE#         13
  C:26AAH         LINE#         14
  C:26AEH         LINE#         15
  C:26B8H         LINE#         16
  C:26BDH         LINE#         17
  C:26BFH         LINE#         19
  -------         ENDPROC       _DELAYMS
  -------         PROC          INITIAL_TRIM
  -------         DO            
  D:0007H         SYMBOL        temp
  -------         ENDDO         
  C:2460H         LINE#         27
  C:2460H         LINE#         28
  C:2460H         LINE#         31
  C:2465H         LINE#         32
  C:2467H         LINE#         33
  C:246DH         LINE#         34
  C:2471H         LINE#         35
  C:2475H         LINE#         37
  C:247BH         LINE#         38
  C:2481H         LINE#         39
  C:2485H         LINE#         40
  C:2489H         LINE#         42
  C:248FH         LINE#         43
  C:2495H         LINE#         44
  C:2499H         LINE#         45
  C:249DH         LINE#         47
  C:24A3H         LINE#         48
  C:24A9H         LINE#         49
BL51 BANKED LINKER/LOCATER V6.22                                                      08/01/2023  15:41:50  PAGE 8


  C:24ADH         LINE#         50
  C:24B1H         LINE#         51
  C:24B7H         LINE#         52
  -------         ENDPROC       INITIAL_TRIM
  -------         PROC          SYSTEM_INIT
  C:0066H         LINE#         60
  C:0066H         LINE#         61
  C:0066H         LINE#         62
  C:006CH         LINE#         76
  C:006FH         LINE#         88
  C:0072H         LINE#         113
  C:0078H         LINE#         114
  C:007FH         LINE#         115
  -------         ENDPROC       SYSTEM_INIT
  -------         ENDMOD        INITIAL

  -------         MODULE        MAIN
  C:0000H         SYMBOL        _ICE_DUMMY_
  D:00A8H         PUBLIC        IE
  C:2163H         PUBLIC        KeyProcess
  B:0080H.1       PUBLIC        P0_1
  B:0090H.1       PUBLIC        P1_1
  B:0080H.3       PUBLIC        P0_3
  B:00B0H.1       PUBLIC        P3_1
  B:00A0H.2       PUBLIC        P2_2
  B:0080H.6       PUBLIC        P0_6
  B:0090H.6       PUBLIC        P1_6
  B:00A0H.7       PUBLIC        P2_7
  C:232FH         PUBLIC        main
  D:00E0H         PUBLIC        ACC
  D:00F8H         PUBLIC        SLPTIM_CR
  B:00A8H.7       PUBLIC        IE_EA
  D:0080H         PUBLIC        P0_DR
  D:0090H         PUBLIC        P1_DR
  D:00A0H         PUBLIC        P2_DR
  D:00B0H         PUBLIC        P3_DR
  D:00D0H         PUBLIC        PSW
  -------         PROC          KEYPROCESS
  -------         DO            
  D:0009H         SYMBOL        key
  -------         ENDDO         
  C:2163H         LINE#         31
  C:2163H         LINE#         32
  C:2163H         LINE#         33
  C:216EH         LINE#         36
  C:217CH         LINE#         37
  C:218AH         LINE#         38
  C:2198H         LINE#         39
  C:21A6H         LINE#         40
  C:21B4H         LINE#         41
  C:21C2H         LINE#         42
  C:21D0H         LINE#         43
  C:21DEH         LINE#         44
  -------         ENDPROC       KEYPROCESS
  -------         PROC          MAIN
  -------         DO            
  D:0008H         SYMBOL        i
BL51 BANKED LINKER/LOCATER V6.22                                                      08/01/2023  15:41:50  PAGE 9


  -------         ENDDO         
  C:232FH         LINE#         47
  C:232FH         LINE#         48
  C:232FH         LINE#         51
  C:2332H         LINE#         52
  C:2335H         LINE#         53
  C:2338H         LINE#         54
  C:2355H         LINE#         56
  C:2358H         LINE#         57
  C:2358H         LINE#         58
  C:235FH         LINE#         59
  C:2361H         LINE#         60
  C:2363H         LINE#         61
  C:2365H         LINE#         62
  C:2367H         LINE#         63
  C:2369H         LINE#         64
  C:236BH         LINE#         65
  C:236DH         LINE#         66
  C:236FH         LINE#         67
  C:2376H         LINE#         68
  C:2378H         LINE#         69
  C:237AH         LINE#         70
  C:237CH         LINE#         71
  C:237EH         LINE#         72
  C:2380H         LINE#         73
  C:2382H         LINE#         74
  C:2384H         LINE#         75
  C:2386H         LINE#         76
  C:238FH         LINE#         78
  C:2391H         LINE#         80
  C:2391H         LINE#         81
  C:2391H         LINE#         82
  C:2394H         LINE#         83
  C:2397H         LINE#         84
  -------         ENDPROC       MAIN
  -------         ENDMOD        MAIN

  -------         MODULE        TOUCHKEYSCAN
  C:0000H         SYMBOL        _ICE_DUMMY_
  D:00A8H         PUBLIC        IE
  C:23F9H         PUBLIC        DeepSleepCfg
  D:00FAH         PUBLIC        SLPTIM_CLR
  C:2706H         PUBLIC        Timer0_Init
  D:0089H         PUBLIC        TMOD
  D:0088H         PUBLIC        TCON
  C:005CH         PUBLIC        WDT_IRQ
  C:255DH         PUBLIC        Timer0_IRQHandler
  D:00E0H         PUBLIC        ACC
  X:0000H         PUBLIC        ChnInfoBuf
  C:2399H         PUBLIC        TKChnCfg
  D:008CH         PUBLIC        TH0
  D:008AH         PUBLIC        TL0
  D:00F8H         PUBLIC        SLPTIM_CR
  D:00F9H         PUBLIC        SLPTIM_SR
  C:25A1H         PUBLIC        CSD_IRQHandler
  D:008EH         PUBLIC        CKCON
  D:0080H         PUBLIC        P0_DR
BL51 BANKED LINKER/LOCATER V6.22                                                      08/01/2023  15:41:50  PAGE 10


  D:0090H         PUBLIC        P1_DR
  D:00A0H         PUBLIC        P2_DR
  D:00B0H         PUBLIC        P3_DR
  D:00D0H         PUBLIC        PSW
  -------         PROC          TIMER0_IRQHANDLER
  C:255DH         LINE#         31
  C:257AH         LINE#         33
  C:257DH         LINE#         34
  C:2580H         LINE#         35
  C:2583H         LINE#         37
  C:2586H         LINE#         38
  -------         ENDPROC       TIMER0_IRQHANDLER
  -------         PROC          CSD_IRQHANDLER
  C:25A1H         LINE#         41
  C:25BEH         LINE#         43
  C:25C1H         LINE#         44
  -------         ENDPROC       CSD_IRQHANDLER
  -------         PROC          WDT_IRQ
  C:005CH         LINE#         47
  C:005CH         LINE#         49
  C:005FH         LINE#         50
  C:0062H         LINE#         51
  -------         ENDPROC       WDT_IRQ
  -------         PROC          TIMER0_INIT
  C:2706H         LINE#         54
  C:2706H         LINE#         55
  C:2706H         LINE#         56
  C:2709H         LINE#         57
  C:270CH         LINE#         58
  C:270FH         LINE#         59
  C:2712H         LINE#         60
  C:2715H         LINE#         61
  -------         ENDPROC       TIMER0_INIT
  -------         ENDMOD        TOUCHKEYSCAN

  -------         MODULE        TOUCH_LIB
  C:0000H         SYMBOL        _ICE_DUMMY_
  C:1CACH         PUBLIC        _TKL_Key_CalibrationTreatment
  C:1F27H         PUBLIC        TKL_ScanStartLoop
  C:2716H         PUBLIC        WDT_init
  C:1B5AH         SYMBOL        _TKL_Key_SetIdleState
  D:00A8H         PUBLIC        IE
  C:2675H         SYMBOL        _TKL_Key_SetPostDetectState
  C:25DCH         SYMBOL        _TKL_Key_SetPreDetectState
  C:1E8EH         SYMBOL        _TKL_Key_IdleTreatment
  C:2401H         SYMBOL        _TKL_Key_SetErrorState
  C:1DF4H         SYMBOL        _TKL_Key_SetFindIcomState
  C:19D8H         PUBLIC        TKL_GetKeyValue
  D:00FAH         PUBLIC        SLPTIM_CLR
  C:08A2H         SYMBOL        _TKL_Key_FindIcomTreatment
  C:2252H         SYMBOL        _TKL_Key_SetPreCalibrationState
  C:0D3EH         SYMBOL        TKL_ECS
  C:22C2H         SYMBOL        _TKL_Key_PreCalibrationTreatment
  C:26C0H         PUBLIC        TKL_Action
  C:18C5H         SYMBOL        _TKL_AddDataToBuf
  C:1D52H         SYMBOL        _TKL_Key_DetectedTreatment
  C:0036H         PUBLIC        TKL_CSDInit
BL51 BANKED LINKER/LOCATER V6.22                                                      08/01/2023  15:41:50  PAGE 11


  D:00FFH         PUBLIC        SLPTIM_PRDRH
  D:0092H         PUBLIC        SCR_SLEEP
  C:0003H         SYMBOL        _TKL_Key_CheckError
  D:00E0H         PUBLIC        ACC
  C:062DH         PUBLIC        _ThresholdInit
  C:1AA2H         SYMBOL        TKL_ProcessAll
  C:2048H         PUBLIC        TKL_IRQCallback
  C:24B8H         SYMBOL        _TKL_Key_DeltaCaculation
  C:26D8H         SYMBOL        _TKL_Key_BackIdleState
  D:00F8H         PUBLIC        SLPTIM_CR
  C:14E1H         SYMBOL        TKL_WaterProof
  C:135CH         SYMBOL        _TKL_Acquisition
  D:00F9H         PUBLIC        SLPTIM_SR
  C:1189H         PUBLIC        _TKL_Init
  C:1790H         SYMBOL        _TKL_Key_PostDetectedTreatment
  C:1654H         SYMBOL        _TKL_Key_PreDetectedTreatment
  C:1FB8H         SYMBOL        _TKL_Key_SetDetectState
  C:0FBDH         SYMBOL        _gpio_set_mode
  C:26EFH         SYMBOL        _TKL_Key_BackToDetectState
  C:2629H         PUBLIC        _Delay
  C:1C05H         SYMBOL        _TKL_scan
  D:0080H         PUBLIC        P0_DR
  D:0090H         PUBLIC        P1_DR
  C:2643H         SYMBOL        TKL_AcquisitionAll
  D:00A0H         PUBLIC        P2_DR
  D:00B0H         PUBLIC        P3_DR
  D:0029H         PUBLIC        TKLInfo
  C:21DFH         SYMBOL        _TKL_Key_SetCalibrationState
  D:00D0H         PUBLIC        PSW
  -------         PROC          L?0278
  -------         ENDPROC       L?0278
  -------         PROC          _DELAY
  D:0006H         SYMBOL        ms
  -------         DO            
  D:0004H         SYMBOL        a
  -------         ENDDO         
  C:2629H         LINE#         182
  C:2629H         LINE#         183
  C:2629H         LINE#         185
  C:262DH         LINE#         186
  C:262DH         LINE#         187
  C:2631H         LINE#         188
  C:263BH         LINE#         189
  C:2640H         LINE#         190
  C:2642H         LINE#         192
  -------         ENDPROC       _DELAY
  -------         PROC          TKL_CSDINIT
  C:0036H         LINE#         200
  C:0036H         LINE#         201
  C:0036H         LINE#         203
  C:003DH         LINE#         204
  C:0042H         LINE#         205
  C:0047H         LINE#         208
  C:004DH         LINE#         209
  C:0053H         LINE#         210
  C:0057H         LINE#         211
  C:005BH         LINE#         216
BL51 BANKED LINKER/LOCATER V6.22                                                      08/01/2023  15:41:50  PAGE 12


  -------         ENDPROC       TKL_CSDINIT
  -------         PROC          _THRESHOLDINIT
  D:001DH         SYMBOL        chn
  D:001EH         SYMBOL        cfg
  C:062DH         LINE#         219
  C:0635H         LINE#         220
  C:0635H         LINE#         221
  C:0655H         LINE#         222
  C:0682H         LINE#         223
  C:06A8H         LINE#         225
  C:06C9H         LINE#         226
  C:071EH         LINE#         227
  C:074BH         LINE#         229
  C:079FH         LINE#         230
  C:07CCH         LINE#         231
  C:081BH         LINE#         233
  C:0831H         LINE#         234
  C:0847H         LINE#         236
  C:0858H         LINE#         237
  C:0869H         LINE#         239
  C:0897H         LINE#         241
  -------         ENDPROC       _THRESHOLDINIT
  -------         PROC          _TKL_ADDDATATOBUF
  D:0027H         SYMBOL        dat
  C:18C5H         LINE#         251
  C:18C9H         LINE#         252
  C:18C9H         LINE#         254
  C:18CEH         LINE#         255
  C:18CEH         LINE#         256
  C:1938H         LINE#         257
  C:1938H         LINE#         258
  C:1964H         LINE#         259
  C:1998H         LINE#         262
  C:19A8H         LINE#         263
  C:19A8H         LINE#         264
  C:19BFH         LINE#         266
  C:19C4H         LINE#         267
  C:19C4H         LINE#         269
  C:19C7H         LINE#         270
  C:19C8H         LINE#         271
  C:19D1H         LINE#         272
  C:19D1H         LINE#         274
  C:19D4H         LINE#         275
  C:19D7H         LINE#         276
  C:19D7H         LINE#         277
  C:19D7H         LINE#         278
  -------         ENDPROC       _TKL_ADDDATATOBUF
  -------         PROC          TKL_SCANSTARTLOOP
  C:1F27H         LINE#         285
  C:1F27H         LINE#         286
  C:1F27H         LINE#         287
  C:1F2FH         LINE#         290
  C:1F3CH         LINE#         291
  C:1F3CH         LINE#         292
  C:1F3EH         LINE#         293
  C:1F44H         LINE#         294
  C:1F44H         LINE#         295
BL51 BANKED LINKER/LOCATER V6.22                                                      08/01/2023  15:41:50  PAGE 13


  C:1F46H         LINE#         296
  C:1F4EH         LINE#         297
  C:1F4EH         LINE#         298
  C:1F58H         LINE#         299
  C:1F58H         LINE#         300
  C:1F5DH         LINE#         301
  C:1F60H         LINE#         302
  C:1F60H         LINE#         303
  C:1F6BH         LINE#         304
  C:1F6BH         LINE#         305
  C:1F73H         LINE#         306
  C:1F73H         LINE#         307
  C:1F73H         LINE#         313
  C:1F88H         LINE#         314
  C:1F88H         LINE#         316
  C:1F88H         LINE#         319
  C:1F96H         LINE#         322
  C:1F9CH         LINE#         328
  C:1FA2H         LINE#         329
  C:1FA7H         LINE#         330
  C:1FABH         LINE#         332
  C:1FB1H         LINE#         337
  C:1FB7H         LINE#         342
  -------         ENDPROC       TKL_SCANSTARTLOOP
  -------         PROC          TKL_IRQCALLBACK
  C:2048H         LINE#         349
  C:2048H         LINE#         350
  C:2048H         LINE#         352
  C:204EH         LINE#         354
  C:205DH         LINE#         355
  C:205DH         LINE#         357
  C:2064H         LINE#         358
  C:2064H         LINE#         359
  C:2064H         LINE#         360
  C:2067H         LINE#         362
  C:2067H         LINE#         364
  C:206AH         LINE#         367
  C:206EH         LINE#         368
  C:206EH         LINE#         369
  C:206EH         LINE#         370
  C:2071H         LINE#         371
  C:2071H         LINE#         372
  C:2071H         LINE#         373
  C:2074H         LINE#         375
  C:2074H         LINE#         377
  C:207FH         LINE#         380
  C:20A0H         LINE#         383
  C:20ADH         LINE#         384
  C:20BEH         LINE#         385
  C:20BEH         LINE#         387
  C:20CBH         LINE#         388
  C:20CCH         LINE#         390
  C:20CCH         LINE#         392
  C:20CDH         LINE#         393
  C:20CDH         LINE#         394
  C:20CDH         LINE#         395
  C:20D0H         LINE#         396
BL51 BANKED LINKER/LOCATER V6.22                                                      08/01/2023  15:41:50  PAGE 14


  C:20D6H         LINE#         397
  C:20D6H         LINE#         398
  C:20D6H         LINE#         399
  -------         ENDPROC       TKL_IRQCALLBACK
  -------         PROC          _TKL_ACQUISITION
  D:000AH         SYMBOL        Chn
  D:000BH         SYMBOL        pMeasurement
  -------         DO            
  D:000EH         SYMBOL        dat
  D:0010H         SYMBOL        Max1
  D:0012H         SYMBOL        Max2
  D:0014H         SYMBOL        Min1
  D:0016H         SYMBOL        Min2
  D:0018H         SYMBOL        Sampling
  D:0004H         SYMBOL        tmpval
  D:0019H         SYMBOL        MaxMeasurement
  D:001BH         SYMBOL        MinMeasurement
  -------         ENDDO         
  C:135CH         LINE#         410
  C:1364H         LINE#         411
  C:1364H         LINE#         415
  C:1377H         LINE#         420
  C:137CH         LINE#         421
  C:1380H         LINE#         423
  C:1390H         LINE#         424
  C:1390H         LINE#         425
  C:13B3H         LINE#         428
  C:13B7H         LINE#         429
  C:13B7H         LINE#         430
  C:13C2H         LINE#         431
  C:13D0H         LINE#         432
  C:13DBH         LINE#         433
  C:13EAH         LINE#         434
  C:13ECH         LINE#         436
  C:1402H         LINE#         437
  C:1402H         LINE#         438
  C:1426H         LINE#         439
  C:1429H         LINE#         440
  C:1429H         LINE#         442
  C:1434H         LINE#         443
  C:1434H         LINE#         444
  C:143AH         LINE#         445
  C:1440H         LINE#         446
  C:1442H         LINE#         447
  C:144DH         LINE#         448
  C:144DH         LINE#         449
  C:1453H         LINE#         450
  C:1453H         LINE#         451
  C:145EH         LINE#         452
  C:145EH         LINE#         453
  C:1464H         LINE#         454
  C:146AH         LINE#         455
  C:146CH         LINE#         456
  C:1477H         LINE#         457
  C:1477H         LINE#         458
  C:147DH         LINE#         459
  C:147DH         LINE#         460
BL51 BANKED LINKER/LOCATER V6.22                                                      08/01/2023  15:41:50  PAGE 15


  C:1482H         LINE#         461
  C:14BEH         LINE#         462
  C:14DEH         LINE#         464
  C:14E0H         LINE#         465
  -------         ENDPROC       _TKL_ACQUISITION
  -------         PROC          TKL_ACQUISITIONALL
  -------         DO            
  D:0009H         SYMBOL        chn
  -------         ENDDO         
  C:2643H         LINE#         471
  C:2643H         LINE#         472
  C:2643H         LINE#         476
  C:2654H         LINE#         477
  C:2654H         LINE#         478
  C:2670H         LINE#         479
  C:2674H         LINE#         480
  -------         ENDPROC       TKL_ACQUISITIONALL
  -------         PROC          _TKL_KEY_DELTACACULATION
  D:000AH         SYMBOL        chn
  C:24B8H         LINE#         488
  C:24BAH         LINE#         489
  C:24BAH         LINE#         490
  C:24D9H         LINE#         491
  C:24D9H         LINE#         493
  C:24E2H         LINE#         494
  C:24E4H         LINE#         496
  C:24E4H         LINE#         497
  C:250AH         LINE#         498
  C:250AH         LINE#         499
  -------         ENDPROC       _TKL_KEY_DELTACACULATION
  -------         PROC          _TKL_KEY_SETFINDICOMSTATE
  D:001DH         SYMBOL        chn
  C:1DF4H         LINE#         506
  C:1DF6H         LINE#         507
  C:1DF6H         LINE#         508
  C:1E0EH         LINE#         509
  C:1E1FH         LINE#         510
  C:1E31H         LINE#         511
  C:1E39H         LINE#         512
  C:1E40H         LINE#         513
  C:1E48H         LINE#         514
  C:1E8DH         LINE#         515
  -------         ENDPROC       _TKL_KEY_SETFINDICOMSTATE
  -------         PROC          _TKL_KEY_SETIDLESTATE
  D:000FH         SYMBOL        chn
  C:1B5AH         LINE#         522
  C:1B5CH         LINE#         523
  C:1B5CH         LINE#         524
  C:1B75H         LINE#         525
  C:1B86H         LINE#         526
  C:1BB8H         LINE#         527
  C:1BBFH         LINE#         528
  C:1C04H         LINE#         529
  -------         ENDPROC       _TKL_KEY_SETIDLESTATE
  -------         PROC          _TKL_KEY_BACKIDLESTATE
  D:0007H         SYMBOL        chn
  C:26D8H         LINE#         536
BL51 BANKED LINKER/LOCATER V6.22                                                      08/01/2023  15:41:50  PAGE 16


  C:26D8H         LINE#         537
  C:26D8H         LINE#         538
  -------         ENDPROC       _TKL_KEY_BACKIDLESTATE
  -------         PROC          _TKL_KEY_SETPREDETECTSTATE
  D:000BH         SYMBOL        chn
  C:25DCH         LINE#         546
  C:25DEH         LINE#         547
  C:25DEH         LINE#         548
  C:25F5H         LINE#         549
  C:2606H         LINE#         550
  C:260DH         LINE#         554
  C:2610H         LINE#         555
  -------         ENDPROC       _TKL_KEY_SETPREDETECTSTATE
  -------         PROC          _TKL_KEY_SETDETECTSTATE
  D:000FH         SYMBOL        chn
  C:1FB8H         LINE#         562
  C:1FBAH         LINE#         563
  C:1FBAH         LINE#         564
  C:1FD3H         LINE#         565
  C:1FE4H         LINE#         566
  C:1FF9H         LINE#         567
  C:2023H         LINE#         568
  C:202AH         LINE#         569
  C:2039H         LINE#         570
  -------         ENDPROC       _TKL_KEY_SETDETECTSTATE
  -------         PROC          _TKL_KEY_BACKTODETECTSTATE
  D:0007H         SYMBOL        chn
  C:26EFH         LINE#         579
  C:26EFH         LINE#         580
  C:26EFH         LINE#         581
  -------         ENDPROC       _TKL_KEY_BACKTODETECTSTATE
  -------         PROC          _TKL_KEY_SETPOSTDETECTSTATE
  D:000BH         SYMBOL        chn
  C:2675H         LINE#         589
  C:2677H         LINE#         590
  C:2677H         LINE#         591
  C:268EH         LINE#         592
  C:269FH         LINE#         593
  -------         ENDPROC       _TKL_KEY_SETPOSTDETECTSTATE
  -------         PROC          _TKL_KEY_SETPRECALIBRATIONSTATE
  D:000BH         SYMBOL        chn
  C:2252H         LINE#         601
  C:2254H         LINE#         602
  C:2254H         LINE#         603
  C:226BH         LINE#         604
  C:227CH         LINE#         605
  C:22C1H         LINE#         606
  -------         ENDPROC       _TKL_KEY_SETPRECALIBRATIONSTATE
  -------         PROC          _TKL_KEY_SETCALIBRATIONSTATE
  D:0024H         SYMBOL        chn
  C:21DFH         LINE#         613
  C:21E1H         LINE#         614
  C:21E1H         LINE#         615
  C:21F8H         LINE#         616
  C:2202H         LINE#         617
  C:220CH         LINE#         618
  C:2251H         LINE#         619
BL51 BANKED LINKER/LOCATER V6.22                                                      08/01/2023  15:41:50  PAGE 17


  -------         ENDPROC       _TKL_KEY_SETCALIBRATIONSTATE
  -------         PROC          _TKL_KEY_SETERRORSTATE
  D:0024H         SYMBOL        chn
  C:2401H         LINE#         626
  C:2403H         LINE#         627
  C:2403H         LINE#         628
  C:241AH         LINE#         629
  C:245FH         LINE#         630
  -------         ENDPROC       _TKL_KEY_SETERRORSTATE
  -------         PROC          _TKL_KEY_CHECKERROR
  D:0007H         SYMBOL        chn
  -------         DO            
  D:0006H         SYMBOL        val
  -------         ENDDO         
  C:0003H         LINE#         649
  C:0003H         LINE#         650
  C:0003H         LINE#         651
  C:001BH         LINE#         652
  C:002CH         LINE#         653
  C:002CH         LINE#         654
  C:002FH         LINE#         655
  C:002FH         LINE#         657
  C:0031H         LINE#         658
  -------         ENDPROC       _TKL_KEY_CHECKERROR
  -------         PROC          _TKL_SCAN
  D:0024H         SYMBOL        chn
  -------         DO            
  D:0025H         SYMBOL        Meas_buff
  -------         ENDDO         
  C:1C05H         LINE#         664
  C:1C07H         LINE#         665
  C:1C07H         LINE#         666
  C:1C0CH         LINE#         668
  C:1C12H         LINE#         674
  C:1C18H         LINE#         675
  C:1C1DH         LINE#         676
  C:1C21H         LINE#         677
  C:1C27H         LINE#         681
  C:1C2DH         LINE#         686
  C:1C35H         LINE#         688
  C:1C3BH         LINE#         689
  C:1C55H         LINE#         690
  C:1C5FH         LINE#         691
  C:1C6BH         LINE#         692
  C:1C71H         LINE#         693
  C:1C77H         LINE#         694
  C:1C7FH         LINE#         695
  C:1C9EH         LINE#         696
  C:1CA8H         LINE#         698
  C:1CABH         LINE#         699
  -------         ENDPROC       _TKL_SCAN
  -------         PROC          _TKL_KEY_FINDICOMTREATMENT
  D:001DH         SYMBOL        chn
  -------         DO            
  D:001EH         SYMBOL        target
  D:0020H         SYMBOL        dat
  -------         ENDDO         
BL51 BANKED LINKER/LOCATER V6.22                                                      08/01/2023  15:41:50  PAGE 18


  C:08A2H         LINE#         706
  C:08A4H         LINE#         707
  C:08A4H         LINE#         708
  C:08AAH         LINE#         709
  C:08B3H         LINE#         711
  C:08D5H         LINE#         712
  C:08D5H         LINE#         713
  C:08DFH         LINE#         714
  C:08DFH         LINE#         715
  C:08F5H         LINE#         716
  C:0911H         LINE#         717
  C:0911H         LINE#         718
  C:092BH         LINE#         719
  C:092BH         LINE#         720
  C:0943H         LINE#         721
  C:0967H         LINE#         722
  C:0967H         LINE#         723
  C:097EH         LINE#         724
  C:097EH         LINE#         725
  C:09B2H         LINE#         726
  C:09B2H         LINE#         727
  C:09C3H         LINE#         728
  C:09C5H         LINE#         730
  C:09C5H         LINE#         731
  C:09DDH         LINE#         732
  C:09F9H         LINE#         733
  C:0A05H         LINE#         734
  C:0A05H         LINE#         736
  C:0A27H         LINE#         737
  C:0A27H         LINE#         738
  C:0A27H         LINE#         739
  C:0A2AH         LINE#         740
  C:0A2AH         LINE#         741
  C:0A2AH         LINE#         743
  C:0A2AH         LINE#         744
  C:0A59H         LINE#         745
  C:0A59H         LINE#         746
  C:0A72H         LINE#         747
  C:0A77H         LINE#         748
  C:0A77H         LINE#         749
  C:0A77H         LINE#         751
  C:0A77H         LINE#         752
  C:0A94H         LINE#         753
  C:0AB0H         LINE#         754
  C:0ABCH         LINE#         755
  C:0ABCH         LINE#         756
  C:0ACBH         LINE#         757
  C:0ACBH         LINE#         758
  C:0AD0H         LINE#         759
  C:0AD0H         LINE#         760
  C:0AD0H         LINE#         762
  C:0AD0H         LINE#         763
  C:0AD0H         LINE#         764
  C:0AD9H         LINE#         766
  C:0AFAH         LINE#         767
  C:0AFAH         LINE#         768
  C:0AFDH         LINE#         769
BL51 BANKED LINKER/LOCATER V6.22                                                      08/01/2023  15:41:50  PAGE 19


  -------         ENDPROC       _TKL_KEY_FINDICOMTREATMENT
  -------         PROC          _TKL_KEY_IDLETREATMENT
  D:000AH         SYMBOL        chn
  -------         DO            
  D:0006H         SYMBOL        th
  -------         ENDDO         
  C:1E8EH         LINE#         776
  C:1E90H         LINE#         777
  C:1E90H         LINE#         780
  C:1EB6H         LINE#         781
  C:1EB6H         LINE#         782
  C:1EBBH         LINE#         784
  C:1EBBH         LINE#         786
  C:1EE2H         LINE#         787
  C:1EF1H         LINE#         788
  C:1EF1H         LINE#         789
  C:1EF6H         LINE#         791
  C:1EF6H         LINE#         794
  C:1F10H         LINE#         795
  C:1F10H         LINE#         796
  C:1F26H         LINE#         797
  C:1F26H         LINE#         798
  -------         ENDPROC       _TKL_KEY_IDLETREATMENT
  -------         PROC          _TKL_KEY_PREDETECTEDTREATMENT
  D:000AH         SYMBOL        chn
  -------         DO            
  D:000BH         SYMBOL        preth
  D:000DH         SYMBOL        th
  -------         ENDDO         
  C:1654H         LINE#         805
  C:1656H         LINE#         806
  C:1656H         LINE#         807
  C:1680H         LINE#         808
  C:16BBH         LINE#         810
  C:16D6H         LINE#         811
  C:16D6H         LINE#         812
  C:16F5H         LINE#         813
  C:16F5H         LINE#         815
  C:1706H         LINE#         816
  C:1706H         LINE#         818
  C:1720H         LINE#         819
  C:1720H         LINE#         820
  C:1736H         LINE#         821
  C:1736H         LINE#         822
  C:1754H         LINE#         823
  C:1754H         LINE#         824
  C:1759H         LINE#         825
  C:1759H         LINE#         826
  C:1759H         LINE#         827
  C:176AH         LINE#         828
  C:176AH         LINE#         829
  C:176FH         LINE#         830
  C:176FH         LINE#         831
  C:178AH         LINE#         832
  C:178AH         LINE#         834
  C:178FH         LINE#         835
  C:178FH         LINE#         836
BL51 BANKED LINKER/LOCATER V6.22                                                      08/01/2023  15:41:50  PAGE 20


  -------         ENDPROC       _TKL_KEY_PREDETECTEDTREATMENT
  -------         PROC          _TKL_KEY_DETECTEDTREATMENT
  D:000AH         SYMBOL        chn
  -------         DO            
  D:0006H         SYMBOL        th
  -------         ENDDO         
  C:1D52H         LINE#         843
  C:1D54H         LINE#         844
  C:1D54H         LINE#         845
  C:1D7AH         LINE#         847
  C:1D89H         LINE#         848
  C:1D89H         LINE#         849
  C:1D8EH         LINE#         851
  C:1D8EH         LINE#         854
  C:1D94H         LINE#         855
  C:1D94H         LINE#         856
  C:1DBEH         LINE#         857
  C:1DBEH         LINE#         858
  C:1DC3H         LINE#         860
  C:1DC3H         LINE#         861
  C:1DC3H         LINE#         864
  C:1DDDH         LINE#         865
  C:1DDDH         LINE#         866
  C:1DF3H         LINE#         867
  C:1DF3H         LINE#         868
  -------         ENDPROC       _TKL_KEY_DETECTEDTREATMENT
  -------         PROC          _TKL_KEY_POSTDETECTEDTREATMENT
  D:000AH         SYMBOL        chn
  -------         DO            
  D:000BH         SYMBOL        preth
  D:000DH         SYMBOL        th
  -------         ENDDO         
  C:1790H         LINE#         875
  C:1792H         LINE#         876
  C:1792H         LINE#         877
  C:17BCH         LINE#         878
  C:17F7H         LINE#         880
  C:1812H         LINE#         881
  C:1812H         LINE#         882
  C:1831H         LINE#         883
  C:1831H         LINE#         885
  C:1842H         LINE#         886
  C:1842H         LINE#         887
  C:185CH         LINE#         888
  C:185CH         LINE#         889
  C:1872H         LINE#         890
  C:1872H         LINE#         891
  C:188CH         LINE#         892
  C:188CH         LINE#         893
  C:188CH         LINE#         894
  C:188CH         LINE#         895
  C:188EH         LINE#         896
  C:189FH         LINE#         897
  C:189FH         LINE#         898
  C:18A4H         LINE#         899
  C:18A4H         LINE#         900
  C:18BFH         LINE#         901
BL51 BANKED LINKER/LOCATER V6.22                                                      08/01/2023  15:41:50  PAGE 21


  C:18BFH         LINE#         903
  C:18C4H         LINE#         904
  C:18C4H         LINE#         905
  -------         ENDPROC       _TKL_KEY_POSTDETECTEDTREATMENT
  -------         PROC          _TKL_KEY_PRECALIBRATIONTREATMENT
  D:000AH         SYMBOL        chn
  C:22C2H         LINE#         912
  C:22C4H         LINE#         913
  C:22C4H         LINE#         914
  C:22EAH         LINE#         915
  C:22EAH         LINE#         916
  C:22F4H         LINE#         917
  C:22F4H         LINE#         918
  C:230AH         LINE#         919
  C:230AH         LINE#         920
  C:2324H         LINE#         921
  C:2324H         LINE#         922
  C:2329H         LINE#         923
  C:2329H         LINE#         924
  C:2329H         LINE#         926
  C:2329H         LINE#         927
  C:232EH         LINE#         928
  C:232EH         LINE#         929
  -------         ENDPROC       _TKL_KEY_PRECALIBRATIONTREATMENT
  -------         PROC          _TKL_KEY_CALIBRATIONTREATMENT
  D:000AH         SYMBOL        chn
  C:1CACH         LINE#         936
  C:1CAEH         LINE#         937
  C:1CAEH         LINE#         938
  C:1D06H         LINE#         939
  C:1D20H         LINE#         940
  C:1D2AH         LINE#         941
  C:1D2AH         LINE#         942
  C:1D4CH         LINE#         943
  C:1D51H         LINE#         944
  C:1D51H         LINE#         945
  -------         ENDPROC       _TKL_KEY_CALIBRATIONTREATMENT
  -------         PROC          TKL_PROCESSALL
  -------         DO            
  D:0009H         SYMBOL        chn
  -------         ENDDO         
  C:1AA2H         LINE#         952
  C:1AA2H         LINE#         953
  C:1AA2H         LINE#         956
  C:1AA6H         LINE#         957
  C:1AA6H         LINE#         958
  C:1AA8H         LINE#         959
  C:1AA8H         LINE#         961
  C:1ABCH         LINE#         962
  C:1ABCH         LINE#         971
  C:1AC1H         LINE#         974
  C:1B00H         LINE#         975
  C:1B00H         LINE#         976
  C:1B00H         LINE#         977
  C:1B0AH         LINE#         978
  C:1B0AH         LINE#         979
  C:1B0AH         LINE#         980
BL51 BANKED LINKER/LOCATER V6.22                                                      08/01/2023  15:41:50  PAGE 22


  C:1B0CH         LINE#         981
  C:1B0CH         LINE#         982
  C:1B0FH         LINE#         983
  C:1B11H         LINE#         984
  C:1B11H         LINE#         985
  C:1B16H         LINE#         986
  C:1B18H         LINE#         987
  C:1B18H         LINE#         988
  C:1B22H         LINE#         989
  C:1B22H         LINE#         990
  C:1B22H         LINE#         991
  C:1B24H         LINE#         992
  C:1B24H         LINE#         993
  C:1B27H         LINE#         994
  C:1B29H         LINE#         995
  C:1B29H         LINE#         996
  C:1B2EH         LINE#         997
  C:1B30H         LINE#         998
  C:1B30H         LINE#         999
  C:1B35H         LINE#         1000
  C:1B37H         LINE#         1001
  C:1B37H         LINE#         1002
  C:1B41H         LINE#         1003
  C:1B41H         LINE#         1004
  C:1B44H         LINE#         1005
  C:1B46H         LINE#         1006
  C:1B46H         LINE#         1007
  C:1B49H         LINE#         1008
  C:1B4BH         LINE#         1009
  C:1B4BH         LINE#         1010
  C:1B50H         LINE#         1011
  C:1B52H         LINE#         1012
  C:1B52H         LINE#         1013
  C:1B52H         LINE#         1014
  C:1B52H         LINE#         1016
  C:1B54H         LINE#         1017
  C:1B54H         LINE#         1018
  C:1B54H         LINE#         1019
  C:1B59H         LINE#         1020
  -------         ENDPROC       TKL_PROCESSALL
  -------         PROC          TKL_WATERPROOF
  -------         DO            
  D:0009H         SYMBOL        chn
  D:000AH         SYMBOL        cnt
  D:000BH         SYMBOL        maxId
  D:000CH         SYMBOL        max1st
  D:000DH         SYMBOL        max2nd
  D:000EH         SYMBOL        percent
  D:000FH         SYMBOL        val
  -------         ENDDO         
  C:14E1H         LINE#         1026
  C:14E1H         LINE#         1027
  C:14E1H         LINE#         1028
  C:14E4H         LINE#         1029
  C:14E8H         LINE#         1034
  C:14FBH         LINE#         1035
  C:14FBH         LINE#         1038
BL51 BANKED LINKER/LOCATER V6.22                                                      08/01/2023  15:41:50  PAGE 23


  C:1526H         LINE#         1039
  C:1526H         LINE#         1040
  C:1528H         LINE#         1041
  C:1547H         LINE#         1043
  C:156AH         LINE#         1044
  C:157CH         LINE#         1045
  C:157CH         LINE#         1046
  C:157FH         LINE#         1047
  C:1581H         LINE#         1049
  C:1581H         LINE#         1050
  C:15A2H         LINE#         1051
  C:15A2H         LINE#         1052
  C:15A9H         LINE#         1053
  C:15A9H         LINE#         1054
  C:15ACH         LINE#         1055
  C:15AFH         LINE#         1056
  C:15B2H         LINE#         1057
  C:15B4H         LINE#         1058
  C:15BBH         LINE#         1059
  C:15BBH         LINE#         1060
  C:15BEH         LINE#         1061
  C:15BEH         LINE#         1062
  C:15BEH         LINE#         1063
  C:15C3H         LINE#         1068
  C:15C9H         LINE#         1069
  C:15C9H         LINE#         1070
  C:15F0H         LINE#         1071
  C:15F2H         LINE#         1072
  C:15FDH         LINE#         1073
  C:15FDH         LINE#         1074
  C:1611H         LINE#         1075
  C:1611H         LINE#         1076
  C:1653H         LINE#         1077
  C:1653H         LINE#         1078
  C:1653H         LINE#         1079
  -------         ENDPROC       TKL_WATERPROOF
  -------         PROC          TKL_ECS
  -------         DO            
  D:0009H         SYMBOL        chn
  D:000AH         SYMBOL        K_Filter
  D:000BH         SYMBOL        K_Filter_Complement
  D:000CH         SYMBOL        IIR_Result
  -------         ENDDO         
  C:0D3EH         LINE#         1085
  C:0D3EH         LINE#         1086
  C:0D3EH         LINE#         1092
  C:0D52H         LINE#         1093
  C:0D52H         LINE#         1094
  C:0D75H         LINE#         1095
  C:0D75H         LINE#         1097
  C:0D87H         LINE#         1098
  C:0D8DH         LINE#         1099
  C:0D94H         LINE#         1100
  C:0D94H         LINE#         1101
  C:0DE8H         LINE#         1102
  C:0DFEH         LINE#         1103
  C:0E44H         LINE#         1104
BL51 BANKED LINKER/LOCATER V6.22                                                      08/01/2023  15:41:50  PAGE 24


  C:0E71H         LINE#         1105
  C:0E85H         LINE#         1108
  C:0E92H         LINE#         1109
  C:0E92H         LINE#         1110
  C:0EE1H         LINE#         1111
  C:0EE1H         LINE#         1112
  C:0EF8H         LINE#         1113
  C:0EFAH         LINE#         1115
  C:0EFAH         LINE#         1116
  C:0F14H         LINE#         1117
  C:0F14H         LINE#         1118
  C:0F16H         LINE#         1119
  C:0F54H         LINE#         1120
  C:0F54H         LINE#         1122
  C:0F73H         LINE#         1123
  C:0F73H         LINE#         1124
  C:0F73H         LINE#         1125
  C:0F73H         LINE#         1126
  C:0F78H         LINE#         1127
  -------         ENDPROC       TKL_ECS
  C:0FACH         SYMBOL        L?0277
  -------         PROC          L?0276
  -------         ENDPROC       L?0276
  C:0FACH         SYMBOL        L?0277
  -------         PROC          _GPIO_SET_MODE
  D:0007H         SYMBOL        b_PortPin
  D:0005H         SYMBOL        mode
  C:0FBDH         LINE#         1131
  C:0FBDH         LINE#         1132
  C:0FBDH         LINE#         1133
  C:0FC5H         LINE#         1134
  C:0FC5H         LINE#         1135
  C:0FD2H         LINE#         1136
  C:0FD2H         LINE#         1137
  C:0FE5H         LINE#         1138
  C:0FEBH         LINE#         1139
  C:0FEEH         LINE#         1140
  C:0FF1H         LINE#         1141
  C:1008H         LINE#         1142
  C:1008H         LINE#         1143
  C:101EH         LINE#         1144
  C:1024H         LINE#         1145
  C:1027H         LINE#         1146
  C:1029H         LINE#         1147
  C:1041H         LINE#         1148
  C:1041H         LINE#         1149
  C:105DH         LINE#         1150
  C:1063H         LINE#         1151
  C:1066H         LINE#         1152
  C:1068H         LINE#         1153
  C:1086H         LINE#         1154
  C:1086H         LINE#         1155
  C:109CH         LINE#         1156
  C:10A2H         LINE#         1157
  C:10ADH         LINE#         1158
  C:10ADH         LINE#         1159
  C:10AEH         LINE#         1160
BL51 BANKED LINKER/LOCATER V6.22                                                      08/01/2023  15:41:50  PAGE 25


  C:10B6H         LINE#         1161
  C:10B6H         LINE#         1162
  C:10C3H         LINE#         1163
  C:10C3H         LINE#         1164
  C:10D7H         LINE#         1165
  C:10DDH         LINE#         1166
  C:10E1H         LINE#         1167
  C:10E2H         LINE#         1168
  C:10F9H         LINE#         1169
  C:10F9H         LINE#         1170
  C:1110H         LINE#         1171
  C:1113H         LINE#         1172
  C:1113H         LINE#         1173
  C:1115H         LINE#         1174
  C:112DH         LINE#         1175
  C:112DH         LINE#         1176
  C:114AH         LINE#         1177
  C:114DH         LINE#         1178
  C:114DH         LINE#         1179
  C:114FH         LINE#         1180
  C:1167H         LINE#         1181
  C:1167H         LINE#         1182
  C:117EH         LINE#         1183
  C:1184H         LINE#         1184
  C:1188H         LINE#         1185
  C:1188H         LINE#         1186
  C:1188H         LINE#         1187
  -------         ENDPROC       _GPIO_SET_MODE
  -------         PROC          WDT_INIT
  C:2716H         LINE#         1190
  C:2716H         LINE#         1191
  C:2716H         LINE#         1192
  C:2719H         LINE#         1193
  C:271CH         LINE#         1194
  C:271FH         LINE#         1195
  C:2721H         LINE#         1196
  C:2725H         LINE#         1197
  -------         ENDPROC       WDT_INIT
  -------         PROC          _TKL_INIT
  D:0009H         SYMBOL        p_TKChnCfg
  D:000CH         SYMBOL        ChnNum
  D:000DH         SYMBOL        ChnInfoPtr
  D:0010H         SYMBOL        p_DeepSleepCfg
  -------         DO            
  D:0013H         SYMBOL        chn
  D:0014H         SYMBOL        cfg
  -------         ENDDO         
  C:1189H         LINE#         1206
  C:1191H         LINE#         1207
  C:1191H         LINE#         1211
  C:11A5H         LINE#         1212
  C:11A5H         LINE#         1214
  C:11A5H         LINE#         1217
  C:11AEH         LINE#         1218
  C:11BEH         LINE#         1219
  C:11C1H         LINE#         1221
  C:11CEH         LINE#         1222
BL51 BANKED LINKER/LOCATER V6.22                                                      08/01/2023  15:41:50  PAGE 26


  C:11CEH         LINE#         1223
  C:11E4H         LINE#         1224
  C:1202H         LINE#         1225
  C:1218H         LINE#         1226
  C:1239H         LINE#         1227
  C:1252H         LINE#         1228
  C:1271H         LINE#         1229
  C:127CH         LINE#         1230
  C:1281H         LINE#         1232
  C:128CH         LINE#         1233
  C:1294H         LINE#         1234
  C:129FH         LINE#         1235
  C:12ADH         LINE#         1236
  C:12BDH         LINE#         1237
  C:12E6H         LINE#         1238
  C:130FH         LINE#         1239
  C:1327H         LINE#         1241
  C:1334H         LINE#         1242
  C:1334H         LINE#         1243
  C:1337H         LINE#         1244
  C:1337H         LINE#         1247
  C:133AH         LINE#         1249
  C:1344H         LINE#         1250
  C:1344H         LINE#         1251
  C:1349H         LINE#         1252
  C:134EH         LINE#         1253
  C:1352H         LINE#         1254
  C:1357H         LINE#         1255
  C:135BH         LINE#         1256
  -------         ENDPROC       _TKL_INIT
  -------         PROC          TKL_ACTION
  C:26C0H         LINE#         1262
  C:26C0H         LINE#         1263
  C:26C0H         LINE#         1265
  C:26C8H         LINE#         1266
  C:26C8H         LINE#         1268
  C:26C8H         LINE#         1270
  C:26CBH         LINE#         1271
  C:26CEH         LINE#         1272
  C:26D1H         LINE#         1273
  C:26D4H         LINE#         1276
  C:26D7H         LINE#         1277
  -------         ENDPROC       TKL_ACTION
  -------         PROC          TKL_GETKEYVALUE
  C:19D8H         LINE#         1284
  C:19D8H         LINE#         1285
  C:19D8H         LINE#         1286
  C:19E8H         LINE#         1287
  C:19E8H         LINE#         1288
  C:19FAH         LINE#         1289
  C:19FAH         LINE#         1290
  C:19FDH         LINE#         1291
  C:1A01H         LINE#         1292
  C:1A01H         LINE#         1294
  C:1A0CH         LINE#         1295
  C:1A0CH         LINE#         1296
  C:1A2BH         LINE#         1297
BL51 BANKED LINKER/LOCATER V6.22                                                      08/01/2023  15:41:50  PAGE 27


  C:1A2BH         LINE#         1298
  C:1A2EH         LINE#         1299
  C:1A33H         LINE#         1300
  C:1A36H         LINE#         1301
  C:1A38H         LINE#         1302
  C:1A3CH         LINE#         1303
  C:1A3EH         LINE#         1305
  C:1A3EH         LINE#         1306
  C:1A47H         LINE#         1307
  C:1A47H         LINE#         1309
  C:1A5DH         LINE#         1310
  C:1A5DH         LINE#         1311
  C:1A60H         LINE#         1312
  C:1A61H         LINE#         1313
  C:1A61H         LINE#         1314
  C:1A61H         LINE#         1315
  C:1A61H         LINE#         1317
  C:1A61H         LINE#         1318
  C:1A61H         LINE#         1319
  C:1A61H         LINE#         1320
  C:1A64H         LINE#         1321
  C:1A67H         LINE#         1322
  C:1A6AH         LINE#         1323
  C:1A6AH         LINE#         1324
  C:1A6AH         LINE#         1326
  C:1A8DH         LINE#         1327
  C:1A8DH         LINE#         1328
  C:1A90H         LINE#         1329
  C:1A90H         LINE#         1330
  C:1A90H         LINE#         1331
  C:1A90H         LINE#         1332
  C:1A90H         LINE#         1334
  C:1A90H         LINE#         1335
  C:1A90H         LINE#         1336
  C:1A90H         LINE#         1337
  C:1A93H         LINE#         1338
  C:1A96H         LINE#         1339
  C:1A99H         LINE#         1340
  C:1A99H         LINE#         1341
  C:1A99H         LINE#         1343
  C:1AA1H         LINE#         1344
  -------         ENDPROC       TKL_GETKEYVALUE
  -------         ENDMOD        TOUCH_LIB

  -------         MODULE        ?C?CLDPTR
  C:008EH         PUBLIC        ?C?CLDPTR
  -------         ENDMOD        ?C?CLDPTR

  -------         MODULE        ?C?CLDOPTR
  C:00A7H         PUBLIC        ?C?CLDOPTR
  -------         ENDMOD        ?C?CLDOPTR

  -------         MODULE        ?C?CILDOPTR
  C:00D4H         PUBLIC        ?C?CILDOPTR
  -------         ENDMOD        ?C?CILDOPTR

  -------         MODULE        ?C?CSTPTR
BL51 BANKED LINKER/LOCATER V6.22                                                      08/01/2023  15:41:50  PAGE 28


  C:0107H         PUBLIC        ?C?CSTPTR
  -------         ENDMOD        ?C?CSTPTR

  -------         MODULE        ?C?CSTOPTR
  C:0119H         PUBLIC        ?C?CSTOPTR
  -------         ENDMOD        ?C?CSTOPTR

  -------         MODULE        ?C?SIDIV
  C:013BH         PUBLIC        ?C?SIDIV
  -------         ENDMOD        ?C?SIDIV

  -------         MODULE        ?C?ILDOPTR
  C:0171H         PUBLIC        ?C?ILDOPTR
  -------         ENDMOD        ?C?ILDOPTR

  -------         MODULE        ?C?IILDOPTR
  C:01A9H         PUBLIC        ?C?IILDOPTR
  -------         ENDMOD        ?C?IILDOPTR

  -------         MODULE        ?C?ISTPTR
  C:01F6H         PUBLIC        ?C?ISTPTR
  -------         ENDMOD        ?C?ISTPTR

  -------         MODULE        ?C?ISTOPTR
  C:0215H         PUBLIC        ?C?ISTOPTR
  -------         ENDMOD        ?C?ISTOPTR

  -------         MODULE        ?C?LMUL
  C:0242H         PUBLIC        ?C?LMUL
  -------         ENDMOD        ?C?LMUL

  -------         MODULE        ?C?ULDIV
  C:02CDH         PUBLIC        ?C?ULDIV
  -------         ENDMOD        ?C?ULDIV

  -------         MODULE        ?C?ULCMP
  C:035FH         PUBLIC        ?C?ULCMP
  -------         ENDMOD        ?C?ULCMP

  -------         MODULE        ?C?ULSHR
  C:0370H         PUBLIC        ?C?ULSHR
  -------         ENDMOD        ?C?ULSHR

  -------         MODULE        ?C?LSHL
  C:0383H         PUBLIC        ?C?LSHL
  -------         ENDMOD        ?C?LSHL

  -------         MODULE        ?C?LLDPTR
  C:0396H         PUBLIC        ?C?LLDPTR
  -------         ENDMOD        ?C?LLDPTR

  -------         MODULE        ?C?LLDOPTR
  C:03B6H         PUBLIC        ?C?LLDOPTR
  -------         ENDMOD        ?C?LLDOPTR

  -------         MODULE        ?C?LSTPTR
  C:03E6H         PUBLIC        ?C?LSTPTR
BL51 BANKED LINKER/LOCATER V6.22                                                      08/01/2023  15:41:50  PAGE 29


  -------         ENDMOD        ?C?LSTPTR

  -------         MODULE        ?C?LSTOPTR
  C:0400H         PUBLIC        ?C?LSTOPTR
  -------         ENDMOD        ?C?LSTOPTR

  -------         MODULE        ?C?LLDPTR0
  C:0424H         PUBLIC        ?C?LLDPTR0
  -------         ENDMOD        ?C?LLDPTR0

  -------         MODULE        ?C?LLDOPTR0
  C:0444H         PUBLIC        ?C?LLDOPTR0
  -------         ENDMOD        ?C?LLDOPTR0

  -------         MODULE        ?C?LSTKOPTR
  C:0474H         PUBLIC        ?C?LSTKOPTR
  -------         ENDMOD        ?C?LSTKOPTR

  -------         MODULE        ?C?OFFXADD
  C:0498H         PUBLIC        ?C?OFFXADD
  -------         ENDMOD        ?C?OFFXADD

  -------         MODULE        ?C?LIMUL
  C:04A4H         PUBLIC        ?C?LIMUL
  -------         ENDMOD        ?C?LIMUL

  -------         MODULE        ?C?UIDIV
  C:04D1H         PUBLIC        ?C?UIDIV
  -------         ENDMOD        ?C?UIDIV

  -------         MODULE        ?C?IILDX
  C:0526H         PUBLIC        ?C?IILDX
  -------         ENDMOD        ?C?IILDX

  -------         MODULE        ?C?LLDIDATA
  C:053CH         PUBLIC        ?C?LLDIDATA
  -------         ENDMOD        ?C?LLDIDATA

  -------         MODULE        ?C?LLDXDATA
  C:0548H         PUBLIC        ?C?LLDXDATA
  -------         ENDMOD        ?C?LLDXDATA

  -------         MODULE        ?C?LLDPDATA
  C:0554H         PUBLIC        ?C?LLDPDATA
  -------         ENDMOD        ?C?LLDPDATA

  -------         MODULE        ?C?LLDCODE
  C:0560H         PUBLIC        ?C?LLDCODE
  -------         ENDMOD        ?C?LLDCODE

  -------         MODULE        ?C?LLDIDATA0
  C:0570H         PUBLIC        ?C?LLDIDATA0
  -------         ENDMOD        ?C?LLDIDATA0

  -------         MODULE        ?C?LLDXDATA0
  C:057DH         PUBLIC        ?C?LLDXDATA0
  -------         ENDMOD        ?C?LLDXDATA0
BL51 BANKED LINKER/LOCATER V6.22                                                      08/01/2023  15:41:50  PAGE 30



  -------         MODULE        ?C?LLDPDATA0
  C:0589H         PUBLIC        ?C?LLDPDATA0
  -------         ENDMOD        ?C?LLDPDATA0

  -------         MODULE        ?C?LLDCODE0
  C:0596H         PUBLIC        ?C?LLDCODE0
  -------         ENDMOD        ?C?LLDCODE0

  -------         MODULE        ?C?LSTIDATA
  C:05A6H         PUBLIC        ?C?LSTIDATA
  -------         ENDMOD        ?C?LSTIDATA

  -------         MODULE        ?C?LSTXDATA
  C:05B2H         PUBLIC        ?C?LSTXDATA
  -------         ENDMOD        ?C?LSTXDATA

  -------         MODULE        ?C?LSTPDATA
  C:05BEH         PUBLIC        ?C?LSTPDATA
  -------         ENDMOD        ?C?LSTPDATA

  -------         MODULE        ?C?LSTKIDATA
  C:05CAH         PUBLIC        ?C?LSTKIDATA
  -------         ENDMOD        ?C?LSTKIDATA

  -------         MODULE        ?C?LSTKXDATA
  C:05E3H         PUBLIC        ?C?LSTKXDATA
  -------         ENDMOD        ?C?LSTKXDATA

  -------         MODULE        ?C?LSTKPDATA
  C:0614H         PUBLIC        ?C?LSTKPDATA
  -------         ENDMOD        ?C?LSTKPDATA

Program Size: data=74.0 xdata=536 code=10012
LINK/LOCATE RUN COMPLETE.  0 WARNING(S),  0 ERROR(S)
